S01D000062696E2F6F70656E626C745F73746D3332673037312E7372656394
S315080000000090002079030008C9030008C903000806
S3150800001000000000000000000000000000000000D2
S31508000020000000000000000000000000C9030008EE
S315080000300000000000000000C9030008ED110008D8
S31508000040C9030008C9030008C9030008C903000852
S31508000050C9030008C9030008C9030008C903000842
S31508000060C9030008C9030008C9030008C903000832
S31508000070C9030008C9030008C9030008C903000822
S31508000080C9030008C9030008C9030008C903000812
S31508000090C9030008C9030008C9030008C903000802
S315080000A0C9030008C9030008C9030008C9030008F2
S311080000B0C9030008C9030008C9030008BA
S315080000BC10B5064C2378002B07D1054B002B02D024
S315080000CC044800E000BF0123237010BD3C04002047
S315080000DC0000000048180008044B10B5002B03D08C
S315080000EC0349044800E000BF10BDC04600000000EC
S315080000FC4004002048180008002243088B4274D399
S3150800010C03098B425FD3030A8B4244D3030B8B42FE
S3150800011C28D3030C8B420DD3FF22090212BA030C07
S3150800012C8B4202D31212090265D0030B8B4219D3E8
S3150800013C00E0090AC30B8B4201D3CB03C01A524108
S3150800014C830B8B4201D38B03C01A5241430B8B4250
S3150800015C01D34B03C01A5241030B8B4201D30B0339
S3150800016CC01A5241C30A8B4201D3CB02C01A524160
S3150800017C830A8B4201D38B02C01A5241430A8B4223
S3150800018C01D34B02C01A5241030A8B4201D30B020C
S3150800019CC01A5241CDD2C3098B4201D3CB01C01A26
S315080001AC524183098B4201D38B01C01A5241430930
S315080001BC8B4201D34B01C01A524103098B4201D31E
S315080001CC0B01C01A5241C3088B4201D3CB00C01A8B
S315080001DC524183088B4201D38B00C01A5241430803
S315080001EC8B4201D34B00C01A5241411A00D2014628
S315080001FC524110467047FFE701B5002000F006F89B
S3150800020C02BDC0460029F7D076E770477047C0464E
S3150800021C70B50C4D0C4E761BB61005D0002408CDC7
S3150800022C01349847A642FAD101F008FB074D084E4F
S3150800023C761BB61005D0002408CD01349847A64283
S3150800024CFAD170BDA01A0008A01A0008A01A000856
S3150800025CA81A0008034B10B5002B02D0024800F070
S3150800026C05F810BD000000008902000810B5010051
S3150800027C00230022002000F019F810BD70B5074DB8
S3150800028C074C641BA41005D0013CA300EB589847F7
S3150800029C002CF9D101F0D8FA70BDC046A81A00088E
S315080002ACAC1A00087047C0467047C046F0B5DE4623
S315080002BC45464E465746E0B52A4C83B0050020689D
S315080002CC90469B460E00FFF7EDFF274B1B680193E4
S315080002DCA423019A5B00D258002A38D053682068A8
S315080002EC1F2B3ADC002D0ED1591C02339B00516092
S315080002FC9E50FFF7D9FF002003B03CBC90469946A8
S3150800030CA246AB46F0BD99008946914441468824DD
S3150800031C4F463951C4214900884690444146873C8A
S3150800032C9C400968A24621438C46414664460C60AB
S3150800033C84214C465F4649006750022DD4D11100E2
S3150800034C55468D31FF310C6825430D60CCE7019A73
S3150800035C01994D32FF32CA50C0E7FFF7A5FF0120BD
S3150800036C4042C9E728040020601800080D48854655
S3150800037C002103E00C4B5B58435004310B480C4BE3
S3150800038C42189A42F6D30B4A02E000231360043251
S3150800039C094B9A42F9D300F013F8FFF739FF00F02E
S315080003AC15FCFEE700900020AC1A0008000000209F
S315080003BC3C0400203C04002088090020FEE70000CD
S315080003CC8022024B12059A607047C04600ED00E089
S315080003DCA0220300D20590421AD0134A90420DD09F
S315080003EC124A904218D0124A904219D0114A01204A
S315080003FC93420CD1104B20215A6A02E002210E4B73
S3150800040C5A6A00200A435A625A6A8A435A627047E1
S3150800041C094B01215A6AF4E7074B04215A6AF0E79B
S3150800042C054B08215A6AECE70004005000080050F6
S3150800043C000C00500014005000100240F0B5C646DF
S3150800044C0C6800B54E68002C2ED001230022984665
S3150800045C43469340234023D01D0004685D43A446BD
S3150800046C6C006419E44367466E4327403E430660B6
S3150800047C4E68013E012E07D88668B44667468E68D4
S3150800048C27406E433E438660C668B44667460E6987
S3150800049C3C406E433443C4604E68022E11D00C683F
S315080004AC23000132D340D3D1013E012E05D843682F
S315080004BCCA68A343544323434360002004BC9046B4
S315080004CCF0BD4C69FF2B0AD86D432E01761B65438C
S315080004DC036AB3431D4305624E680C68E0E71B0AC2
S315080004EC5B435B435C43456A1E01F61AB5432E0013
S315080004FC2500354345624E68D1E7C046054B0020BA
S3150800050C5A69002A05DA044A9A60044A9A605869B4
S3150800051CC00F70470020024023016745AB89EFCD19
S3150800052C8022044B120659690A435A615869C0431A
S3150800053CC00F704700200240F8B50700802600F06F
S3150800054C41FE1B4CC519760203E000F03BFEA8429F
S3150800055C21D223693342F8D180212269154BC9056A
S3150800056C1A40A3690B4019001143002B15D1002A18
S3150800057C18D1002918D100F025FE80253F180C4EFD
S3150800058CED0203E000F01EFE874204D933692B42C4
S3150800059CF8D1002000E00320F8BDA0690343A3614D
S315080005AC002A01D0024B1A61034B01205960F3E76C
S315080005BC00200240FAC3000058040020F0B5C646D5
S315080005CC00B5224E9846337807000D001400012B0F
S315080005DC31D00123FA203370002380007360FFF7B3
S315080005ECABFF002822D11A4A012F26D08023516945
S315080005FCDB020B435361EFF3108072B6631CFF33B7
S3150800060C2D1B22682A510434A342FAD180221049A0
S3150800061C52020B691342FCD180F31088FA20800031
S3150800062CFFF78AFF0A4A5369BB43536100233370A9
S3150800063C04BC9046F0BD0220FAE753693B4353616C
S3150800064C2C60BFF36F8F43466B60E7E758040020B6
S3150800065C002002408022164B520019680A4380215A
S3150800066C1A60C9001A680A42FCD05A681149114026
S3150800067C8022D2010A435A60002280219A600132F4
S3150800068CFF321A600A4B89021A680A42FCD1802288
S3150800069C802152001A60064A890413680B40FCD163
S315080006AC80214901D1609361013B00201362704798
S315080006BC00100240FF80FFFF032010B50D4AD368D7
S315080006CC18400338431E98410B4B40429C46184031
S315080006DCD368D1685B0449066044D4685B0E490F3D
S315080006EC58430131FFF708FD610F0131FFF704FD8F
S315080006FC10BDC0460010024000127A00382310B50F
S3150800070C084A91680B40082B04D0102B04D1FFF72C
S3150800071CD3FF10BD0448FCE7136804489B045B0F21
S3150800072CD840F6E70010024000127A000024F400C4
S3150800073C70B50400FFF7E2FF1F210A4D2060AB6875
S3150800074C094A1B051B0F9B009A580A40D04060604B
S3150800075CAB68064A5B045B0F9B009B580B40D84062
S3150800076CA06070BD0010024064180008A4180008A8
S3150800077C10B50300032815D000200C2B00D010BD93
S3150800078C234C244A606D0340C02000030343934264
S3150800079C30D0214A934228D0204A934211D1FFF7F0
S315080007ACADFFECE71A4C1E4A606D0340C020800270
S315080007BC034393421ED01B4A934216D01A4A9342BD
S315080007CCEDD0FFF79BFF1F21A268A3681205120F35
S315080007DC164C920012595B040A40D0405B0F144A1F
S315080007EC9B009B580B40D840C9E7E06D8007C00FAB
S315080007FCC003C4E780232068DB00184043425841F5
S3150800080C0C4B404218400C4B9C466044B7E7C0461C
S3150800081C0010024008000C000C000C0004000C0030
S3150800082C020003000300030001000300641800081B
S3150800083CA418000800DC0BFF0024F400F0B5D6461B
S3150800084C4F464646C0B52A4F05003B788A46012BCB
S3150800085C3FD00123FA203B70002380007B60FFF712
S3150800086C6BFE814600282CD12B68042B34D001232F
S3150800087C52465B4213606C68AB68E3189C421BD209
S3150800088C1C4B1D4E984606E0AA686B6894460134C4
S3150800089C6344A34210D94146FA207269E3000A4020
S315080008AC1343164A800013437361FFF745FE00286D
S315080008BCEAD0534681461C6002210F4A53698B4382
S315080008CC536100233B7048461CBC90469946A24689
S315080008DCF0BD02239946F6E7FA20074A084B5169F8
S315080008EC80000B435361FFF727FE8146E9E7C046B4
S315080008FC5804002007FEFFFF0020024002000100FA
S3150800090C04000100F0B50368040085B00D00012051
S3150800091CDB0729D48B68096922680B4369690B4381
S3150800092CE9690B432E490A401343236063682D4A31
S3150800093C1340EA6813436360A3682B4A1340AA69F9
S3150800094C1343A360294B9C4210D0294B9C4233D0AD
S3150800095C284B9C422BD0284B9C4228D02A880F2106
S3150800096CE36A8B431343E36205B0F0BD0230FFF72D
S3150800097CFFFE06002A880120002EF0D06F68002F93
S3150800098CEDD053001D4A3000995AFFF7B5FB80226B
S3150800099CE9697B081202914213D018183900FFF73F
S315080009ACABFB0004000CE0602A880020D7E701A8FE
S315080009BCFFF7BEFE039EDDE70C20FFF7D9FE060007
S315080009CCD8E74000C0183900FFF796FB0C4B0340DC
S315080009DC0007400F1843E0602A880020BFE7C0468E
S315080009ECF369FFEFFFCFFFFFFFFCFFFF0038014065
S315080009FC0044004000480040004C0040C418000861
S31508000A0CF0FF0000FF22032330B51400C5B22B40BB
S31508000A1CDB009C4089010A40E4439A4000280BDB22
S31508000A2C0C4B80089C46C023800060449B00C15830
S31508000A3C0C402243C25030BD0F2307492B408C462D
S31508000A4C083B9B089B006344D9690C402243DA6136
S31508000A5CF1E7C04600E100E000ED00E00A4A431E5B
S31508000A6C012093420ED8C021084A09485360036AEC
S31508000A7C09061B021B0A0B43036200230020936022
S31508000A8C073313607047C046FFFFFF0010E000E015
S31508000A9C00ED00E0014B18607047C0462C0400209E
S31508000AAC0121002210B5074B4942D962DA62196353
S31508000ABC1A6399629A6259625A6200F03DF90020EB
S31508000ACC10BDC0460010024010B50F4B0400196843
S31508000ADC002901D1012010BDFA208000FFF70CFB7C
S31508000AEC0A4B01001868FFF707FBFFF7B7FF00284A
S31508000AFCF0D1032CEED8013800222100FFF782FF33
S31508000B0C034B00201C60E6E7300400202C04002070
S31508000B1C34040020802310B5074A5B0011680020B6
S31508000B2C0B431360FFF7D0FF041E02D001242000EC
S31508000B3C10BD00F0ABF8FAE700200240014B188014
S31508000B4C7047C0467004002010B500F02DFB0E4C03
S31508000B5C236898420FD30D4B1A78002A0CD0002222
S31508000B6C1A70A0232032DB059A6200F01DFB084B95
S31508000B7C1B881B18236010BD01321A70A0231F3264
S31508000B8CDB059A61F1E7C046740400207204002064
S31508000B9C70040020A0232022DB059A627047C04609
S31508000BAC10B5044B00201B699B0402D5FFF7F2FF16
S31508000BBC012010BD0008005010B56420FFF7BEFFD9
S31508000BCC10BDC04610B5FFF7BFFF10BD10B5FFF737
S31508000BDCA1FF0722022025490B68934303430B60A8
S31508000BEC0B681A40022A03D06921214800F0CEF876
S31508000BFC8022204B520019680A431A608022D200C0
S31508000C0C19681142FCD0DA681B4911401B4A0A4381
S31508000C1CDA608022196852040A431A608022D9685D
S31508000C2C52050A43DA608023124A9B04116819425A
S31508000C3CFCD0936812490B409360936811490B409A
S31508000C4C0721936093688B4305390B4393603822CD
S31508000C5C08498B681340102BFBD10B48FFF71AFF7A
S31508000C6C00F0A0F800F0ACF8FCE7C0460020024003
S31508000C7CDC180008001002408C80FF1F3240006010
S31508000C8CFFF0FFFFFF8FFFFF0090D003F0B50125A3
S31508000C9C8020274B8DB01A6C40002A431A641A6CB4
S31508000CACA0262A400592059A996B0024014399635C
S31508000CBC9A6B202702400492049A5A6BF6052A432B
S31508000CCC5A635A6B30002A400392039A0422596BD2
S31508000CDC11435963596B0A4080210292029ADA6BC6
S31508000CEC89020A43DA63DB6B06970B40019306A964
S31508000CFC019B0795089409940A94FFF79FFB802398
S31508000D0CB7629B0106A90B48069307940A94FFF74A
S31508000D1C95FB0C2306A9069330000A3B0793089407
S31508000D2C09940A940B95FFF789FB0DB0F0BDC046E4
S31508000D3C001002400008005010B5A024FFF78AFCEA
S31508000D4C2023E405A3620D48FFF742FB2000FFF7BA
S31508000D5C3FFB0B4B0B49DA6B0B480A400421DA6351
S31508000D6C5A6B8A435A635A6B03398A435A639A6B8A
S31508000D7C02409A631A6C8A431A6410BD0008005024
S31508000D8C00100240FFFFFDFFFFFEFFFF10B500F04D
S31508000D9C05F8FCE710B5FFF70FFF10BD10B5FFF708
S31508000DAC11FF10BD10B500F0F3FCFFF7F3FF00F0D0
S31508000DBCD5F900F023FD00F03DF800F02BF810BD36
S31508000DCC10B5FFF7EBFF00F0E1F900F03FF800F083
S31508000DDC01F810BD10B500F073F8012803D00A4CC1
S31508000DEC2378012B00D010BD00F0DEF9074B084A1A
S31508000DFC1B6812689B18F533FF339842F3D300230C
S31508000E0C237000F0C9FCEEE77C040020780400206F
S31508000E1C800400200122054B10B51A7000F0C4F9A5
S31508000E2C034B1860FFF7D6FF10BDC0467C040020A4
S31508000E3C8004002010B500F04BF800F0E7F900220A
S31508000E4C014B1A7010BDC0463804002010B582B08C
S31508000E5C6B46094CD91D200000F014FA012801D064
S31508000E6C02B010BD0022054B20001A706B46D979CA
S31508000E7C00F04AF8F4E7C046840400203804002041
S31508000E8C7047C04610B5054B1B78002B02D000F0F6
S31508000E9C33F810BDC9B200F0D5F9F8E738040020CC
S31508000EAC044B18780138C3B202209842804140425C
S31508000EBC800170473804002010B5FFF7F1FF10BD0C
S31508000ECC10B500F011F8431E9841C0B210BDC046CB
S31508000EDC00224321034B5A5401319A645A521A8000
S31508000EEC9A707047C4040020024B1878431E984128
S31508000EFCC0B27047C404002043230021014AD154D0
S31508000F0C7047C046C4040020F8B503780500904C19
S31508000F1CFF2B0BD02278012A28D13733DBB2352B9D
S31508000F2C00D900E18B4A9B00D3589F460122E370F7
S31508000F3CEF3B2280A380FFF7B3FFA071FFF7BCFF3E
S31508000F4CE071FFF7B9FF012544230822000A207235
S31508000F5C6572A572E25200F051FC4323E35C012B47
S31508000F6C14D04423E15E002900DDEEE0F8BD00F064
S31508000F7C59FC0028F1D1FE230222E370CD3B2371E4
S31508000F8C1333E2524323E35C012B0ED1FE230222D8
S31508000F9C0221E370EE3B23713433E25243230122E0
S31508000FACE01CE254FFF76EFFE0E74423E15AF5E74D
S31508000FBC00F0F2FBFF230122E370BB3BE252E1E7B0
S31508000FCCFFF76EFF6B780138984200DCB3E0FF231D
S31508000FDC0122E370BB3BE25269780029C7D0AA1CF0
S31508000FECA06C00F00FFC0028C5D0A26C6B78944658
S31508000FFC6344A364B1E74168A06C00F007FC0028C1
S3150800100CD8D1B8E70025FF23A580E370FFF748FF82
S3150800101C00230722E3714423A0712581E252B1E72C
S3150800102CFF23E3704768A66C002F00D18BE00025E0
S3150800103CF71933780136ED18EDB2FFF7AFFEB74264
S3150800104CF7D101230022A3800023E5712272627274
S3150800105C2D0EA37108324433A572E25292E7FFF7BC
S3150800106C1FFF6B78834266D26968201DA1646A7873
S3150800107C00F0B4FBFF23A26CE370944644226B7811
S3150800108C6344A3646B780133A3527BE7FFF708FF2D
S3150800109C6A7890424FD9201DA16CE9E7FE23E370CC
S315080010AC0023022223714433E2526BE7FF23E370D9
S315080010BC0023627823716271E3802372062244232B
S315080010CCE2525FE70023238074E7A66CFFF7E8FE7D
S315080010DC6A1C411E300000F095FB002800D14AE737
S315080010ECFF23E370FFF7DCFEA36C01229C46442326
S315080010FC01386044A064E25244E7FF23E370436876
S3150800110C0122A3644423E2523CE7134B0822A3644E
S3150800111CFF23E370E023DB04636000232381A372BF
S3150800112C4423E2522EE7FE230222E370DE3B2371B0
S3150800113C2433E25226E7FE230222E370DC3B2371BA
S3150800114C2233E2521EE700257BE789B226E7C04622
S3150800115CC4040020E4180008BC1900080022054B3A
S3150800116C05491A60596005219A601960034B1A6083
S3150800117C7047C04610E000E0FFF90000100500209B
S3150800118C0022014B1A60704710E000E0044B1B6804
S3150800119CDB0303D5034A1368013313607047C04653
S315080011AC10E000E010050020044B1A68044B186880
S315080011BCD20301D5013018607047C04610E000E034
S315080011CC10050020044B1A68044B1868D20301D585
S315080011DC013018607047C04610E000E0100500208A
S315080011EC7047C04670B5084C8026A062FFF7DCFF36
S315080011FC0A300500E3691E4205D1FFF7CFFDFFF75C
S3150800120CD3FFA842F6D970BD00440040E12310B5BF
S3150800121C1B0288B001930C220023094C6946200056
S3150800122C0293039304930592069307930093FFF78F
S3150800123C69FB012223681343236008B010BDC0461E
S3150800124C0044004070B506000C008DB240290FD83A
S3150800125C0800FFF7C7FF002D09D00024FFF79EFDF5
S3150800126C305D0134FFF7BEFFA3B29D42F6D870BDC0
S3150800127C74210348FFF78AFD2000FFF7B3FFECE75C
S3150800128CC4190008F8B5204D0E002C78002C16D180
S3150800129C1E4BDA69920602D400242000F8BD5B6A5C
S315080012AC1B4ADBB21370013B3F2BF5D8FFF77CFFCB
S315080012BC184B1860184B1C7001232B70EDE7202473
S315080012CC124AD3691C4015D0134C11492378576A16
S315080012DCCA18577001330A78DBB223709A42DBD1ED
S315080012EC92B2013100F07AFA00232B70237801248C
S315080012FC3370D2E7FFF758FF064B1B6864339842E6
S3150800130CCAD92C70C8E7C0465505002000440040D1
S3150800131C140500205805002056050020F8B50700CE
S3150800132C0D4D00260D4C01E0AC680C35FFF736FD6B
S3150800133CBC4204D82B689C466444BC4204D801368B
S3150800134C0F2EF1D1FF20F8BD73009E19044BB60081
S3150800135C9E19307AF7E7C046F019000800200008F5
S3150800136CEC190008F0B5D64646464F46C0B5804639
S3150800137C0068FFF7D3FF0024FF2805D120001CBC0A
S3150800138C90469946A246F0BDFFF7B8F804234344A5
S3150800139C994680239B0000259A4608E022686368D4
S315080013AC964215D19F4213D10835554514D043465C
S315080013BC1B68EC184B465B191E685F68FFF7EEFC5A
S315080013CC32003B0021000120FFF7F8F80028E5D091
S315080013DC0024FFF7A5F8D1E70124FAE770B5134CFA
S315080013EC05000E00A04214D0114B99420AD123686D
S315080013FCB3420CD02000802240C09200310000F08D
S3150800140CEDF904E0FFF7AEFF0024012806D0200012
S3150800141C70BD084C2368B342F9D0EBE7002DF6D023
S3150800142C2C002368B342F2D0E4E7C04660070020DC
S3150800143C002000085C050020F0B546464F46D64607
S3150800144CC0B599464B0A5B029846036806000C0021
S3150800145C15005A1C35D0984529D10434E41A1E4B6C
S3150800146C34199A4601339C46371DE044A94405E0D5
S3150800147C2B780135237001344D4512D0FFF78EFCBD
S3150800148CE21B5245F4D930004146FFF7A7FF061E6A
S3150800149C15D0071D3C002B780135237001344D45BA
S315080014ACECD101201CBC90469946A246F0BD3000F2
S315080014BC4146FFF793FF061E01D00368CDE70020CF
S315080014CCF0E743460700802208C7920041463800D9
S315080014DC00F084F93368BEE7FF0100000123034AD4
S315080014EC5B421360024A13607047C0465C050020D5
S315080014FC60070020134B70B516004A1E04000D0039
S3150800150C1B1A9A4201D9002070BDFFF707FFFF2866
S3150800151CF9D0601E4019FFF701FFFF28F3D00A4ADD
S3150800152C630A5B02934206D02B003200210007485F
S3150800153CFFF782FFE8E72B00320021000448FFF78B
S3150800154C7BFFE1E7FFFF0108002000085C0500208F
S3150800155C60070020F0B5D6464F464646C0B5504BF8
S3150800156C4A1E86B004000D001B1A9A4207D900249D
S3150800157C200006B01CBC90469946A246F0BDFFF763
S3150800158CCDFE0600601E4019FFF7C8FE0500FF2EAB
S3150800159CEDD0FF28EBD00023002402938642E7D82F
S315080015AC032EE5D91228E3D83E4F0433B84699469C
S315080015BC05E043461B7899460C239C46E044FFF706
S315080015CCEDFB4E4560D00134E4B20F2CF1D1364B0D
S315080015DC9A4601235B429846B9460426002404E041
S315080015EC4B461E780C239C46E144FFF7D7FBB542C5
S315080015FC43D00134E4B20F2CF2D101235B42994655
S3150800160C0426002401E03E780C37FFF7C7FBB542E9
S3150800161C2CD00134E4B20F2CF5D100234A464146AE
S3150800162C551AED1802230393534604930123ED0A26
S3150800163CADB205930024FEF761FF002D08D113E027
S3150800164C049B01340193A4B201330493A5420BD035
S3150800165CFFF7A4FB02A903A8FFF7F0F80028EFD0C0
S3150800166C0024FEF75DFF83E70124FAE763001C19E3
S3150800167C0E4BA4001C196368D0E763001C190B4BAE
S3150800168CA400E3589946BBE763001C19074BA40052
S3150800169CE358F826984636064644F30A9A469BE7D4
S315080016ACFFFF0108001A0008FFFF1E00EC190008CE
S315080016BC00B5104A83B013680120013318D091681D
S315080016CC53688C46D16863448C46116963448C46CE
S315080016DC516963448C46916963448C46D269634468
S315080016EC9B185B4201AA042103480193FFF702FFEA
S315080016FC03B000BD60070020BC2000080D4B18681D
S3150800170C0D4B1B68C0180D4B1B68C0180C4B1B687F
S3150800171CC0180C4B1B68C0180B4B1B68C0180B4B1E
S3150800172C1B68C0180A4B1B68C01843425841C0B204
S3150800173C7047C0460020000804200008082000084E
S3150800174C0C20000810200008142000081820000897
S3150800175CBC20000810B50A48036801330BD10948A8
S3150800176C0368013301D1012010BDFFF7FBFD431EB1
S3150800177C9841C0B2F8E7FFF7F5FD0028F4D0EEE77C
S3150800178C600700205C050020004870470020000810
S3150800179C10B500F04FF810BD10B500F03BF8002856
S315080017AC00D110BDFFF7FCF90028FAD0FFF768FB4B
S315080017BCFFF7E6FCFFF774F900F030F8054B184014
S315080017CC054B986000F02AF8446800F035F8A047F5
S315080017DCE7E7C04680FFFF1F00ED00E070B5002A62
S315080017EC0BD05218461A95B20B784C1C8B55FFF732
S315080017FCD5FAA3B22100AB42F6D170BD10B5FFF7EE
S3150800180C6DFE10BD10B5FFF775FE10BD10B5FFF7D0
S3150800181CA1FE10BD10B5FFF771FF10BD10B5FFF78F
S3150800182CB3FF10BD10B5FFF743FF002801D0FFF733
S3150800183C91FF10BD72B6704762B67047F8B5C046D0
S3150800184CF8BC08BC9E467047F8B5C046F8BC08BC40
S3090800185C9E467047DF
S31508001860000000200000000000000000000000004A
S31508001870000000000000000000000000000000005A
S315080018800000000001000000020000000300000044
S315080018900400000006000000070000000800000021
S315080018A00900000000000000000000000000000021
S315080018B00000000001000000020000000300000014
S315080018C004000000010002000400060008000A00E7
S315080018D00C00100020004000800000016D61696E58
S315080018E02E630000D61000083211000832110008D5
S315080018F0820F00083211000832110008BC0F0008D8
S31508001900CC0F000802100008101000083211000859
S31508001910321100083211000832110008321100088D
S31508001920321100083211000832110008321100087D
S31508001930321100083211000832110008321100086D
S31508001940321100083211000832110008321100085D
S31508001950321100083211000832110008321100084D
S31508001960321100083211000832110008321100083D
S31508001970321100083211000832110008321100082D
S315080019803211000832110008321100082C10000824
S315080019906A1000089810000806110008321100089D
S315080019A03211000832110008161100083211000819
S315080019B0A8100008B8100008D01000084F70656E0F
S315080019C0424C54002E2E2F2E2E2F2E2E2F536F754F
S315080019D07263652F41524D434D305F53544D333238
S315080019E047302F72733233322E630000002000080E
S315080019F00008000004000000002800080008000095
S31508001A00050000000030000800080000060000007D
S31508001A100038000800080000070000000040000821
S31508001A200008000008000000004800080008000040
S31508001A300900000000500008000800000A00000025
S31508001A4000580008000800000B00000000600008AD
S31508001A50000800000C0000000068000800080000EC
S31508001A600D00000000700008000800000E000000CD
S31508001A7000780008000800000F0000000080000839
S31508001A80008000001000000000000108008000002F
S31508001A90110000000080010800800000120000000C
S30D08001AA061020008E5000008D8
S30908001AA8BD00000867
S31508001AAC00000000EC02002054030020BC030020B8
S31508001ABC000000000000000000000000000000000C
S31508001ACC00000000000000000000000000000000FC
S31508001ADC00000000000000000000000000000000EC
S31508001AEC00000000000000000000000000000000DC
S31508001AFC00000000000000000000000000000000CC
S31508001B0C00000000000000000000000000000000BB
S31508001B1C00000000000000000000000000000000AB
S31508001B2C000000000000000000000000000000009B
S31508001B3C000000000000000000000000000000008B
S31508001B4C000000000000000001000000000000007A
S31508001B5C0E33CDAB34126DE6ECDE05000B0000003F
S31508001B6C000000000000000000000000000000005B
S31508001B7C000000000000000000000000000000004B
S31508001B8C000000000000000000000000000000003B
S31508001B9C000000000000000000000000000000002B
S31508001ECC0000000000000000640900200024F40053
S31108001EDC010000000400000004000000E3
S7050800037976
